:100000008FE98DBF1124479A83E088BB83E287B9CB
:1000100083E886B98CE384BB80E690E060E070E022
:1000200040E150E0BBD1809161008F3F11F410920C
:100030006100809162008F3F19F488E7809362002D
:10004000809163008F3F19F482E38093630083E023
:1000500083BF75E0C72E6EE0E62E54E0B52E42E079
:10006000D42E80E690E060E070E040E11FD186B3DE
:100070008170982D990F892B882E8F3F91F700E082
:100080001FEFFF240DD18695811708F4182F08174C
:1000900008F4082FFA94B1F7212F200F802F90E059
:1000A000811B910936E0959587953A95E1F7982F50
:1000B000882309F491E0792E720E622E691A12BE1D
:1000C000552419D118D117D116D115D186B3817005
:1000D000982D990F892B882EC1F7809168009091F7
:1000E0006900A0916A00B0916B000196A11DB11D3D
:1000F0008093680090936900A0936A00B0936B00AE
:100100003998CED0082F399A109162003090610052
:1001100080916000992787FD9095252D30E082170A
:10012000930709F0E8D0612F70E061507040802F94
:1001300090E00ED16FEF70E01DD1162F1F5F389841
:10014000AFD0389A642D70E0809590E001D16BE1DA
:1001500071E010D1062F361608F4362ECCD0882345
:1001600031F484E068E241E071D083E00DC086B3F1
:100170008170982D990F892B882E8F3F41F485E04F
:1001800064E640E063D081E0809364006ACF932D01
:1001900082B78917E8F384D0552019F0681600F16A
:1001A00002C08715E8F0C198BB9AC39A95E0B99A46
:1001B0008E2D8A95F1F7B9988E2D8A95F1F7915089
:1001C000B1F7BB98C398C19A6BD07816C0F1861569
:1001D000B0F150926000302E115009F0B0CF07C03E
:1001E00087E064E141E032D0C09264003ACF1091E0
:1001F000630081D086B38170982D990F892B882E4A
:100200008F3F39F486E064E640E020D0D09264006D
:1002100028CF115071F780916C0090916D00A091E2
:100220006E00B0916F000196A11DB11D80936C000E
:1002300090936D00A0936E00B0936F0012CF83E097
:1002400060E041E003D0B09264000BCF86BF282D60
:10025000E2E47FEF5AE038E7B89AEFBD92E388B75F
:100260008823E9F378BF9150D1F7442389F01FBC6C
:10027000852F8A95F1F7B898832F8A95F1F786B381
:10028000220F8170282B2F3F19F488248A94089517
:10029000662311F3615001F7822E1FBCB8980895B0
:1002A000369A3699FECF85B180950895EF92FF92E8
:1002B0000F931F93CF93DF938C01EB01E42E442324
:1002C00099F0E19911C0F801F080CE0176D08F1538
:1002D00029F0FDBAF894E29AE19A7894EA9421F030
:1002E00021960F5F1F4FEDCFDF91CF911F910F919F
:1002F000FF90EF90089580E690E060E070E040E1CC
:10030000D5DF82B7813E10F080E00895552019F0C6
:10031000C7DF7816B0F7552019F4C2DF861588F7C5
:10032000352D552049F022B7822D90E0820F911D86
:1003300096958795482E02C082B7282E12BEBB9A8A
:100340008CE18A95F1F7BB98532E509481E0089583
:100350005527002480FF02C0060E571F660F771F27
:100360006115710521F096958795009799F7952F5E
:10037000802D0895AA1BBB1B51E107C0AA1FBB1FFC
:10038000A617B70710F0A61BB70B881F991F5A9521
:10039000A9F780959095BC01CD010895A82F862FCF
:1003A000E82FE199FECF1FBA05C0EEBBE09AE395B6
:1003B0000DB20D924150C8F70895E199FECF1FBAD2
:0A03C0008EBBE09A99278DB30895D3
:02000004008278
:020000002AFBD9
:00000001FF
